Component: ARM Compiler 5.06 update 5 (build 528) Tool: armlink [4d35e2]

==============================================================================

Section Cross References

    event_groups.o(.text) refers to heap_1.o(.text) for pvPortMalloc
    event_groups.o(.text) refers to list.o(.text) for vListInitialise
    event_groups.o(.text) refers to tasks.o(.text) for vTaskSuspendAll
    event_groups.o(.text) refers to port.o(.text) for vPortEnterCritical
    queue.o(.text) refers to port.o(.text) for vPortEnterCritical
    queue.o(.text) refers to tasks.o(.text) for xTaskRemoveFromEventList
    queue.o(.text) refers to list.o(.text) for vListInitialise
    queue.o(.text) refers to heap_1.o(.text) for pvPortMalloc
    queue.o(.text) refers to memcpya.o(.text) for __aeabi_memcpy
    tasks.o(.text) refers to list.o(.text) for vListInitialise
    tasks.o(.text) refers to port.o(.text) for vPortEnterCritical
    tasks.o(.text) refers to memseta.o(.text) for __aeabi_memset
    tasks.o(.text) refers to heap_1.o(.text) for pvPortMalloc
    tasks.o(.text) refers to tasks.o(.bss) for pxReadyTasksLists
    tasks.o(.text) refers to tasks.o(.data) for pxDelayedTaskList
    tasks.o(.text) refers to timers.o(.text) for xTimerCreateTimerTask
    tasks.o(.text) refers to main.o(.bss) for ulTaskNumber
    timers.o(.text) refers to list.o(.text) for vListInsert
==============================================================================

Removing Unused input sections from the image.

    Removing event_groups.o(.text), (724 bytes).
    Removing startup_mps_cm3.o(HEAP), (0 bytes).
    Removing dadd.o(.text), (334 bytes).
    Removing dmul.o(.text), (228 bytes).
    Removing ddiv.o(.text), (222 bytes).
    Removing dfixul.o(.text), (48 bytes).
    Removing cdrcmple.o(.text), (48 bytes).
    Removing depilogue.o(.text), (186 bytes).

8 unused section(s) (total 1790 bytes) removed from the image.

==============================================================================

Image Symbol Table

    Local Symbols

    Symbol Name                              Value     Ov Type        Size  Object(Section)

    RESET                                    0x00000000   Section      192  startup_mps_cm3.o(RESET)
    ../clib/microlib/division.c              0x00000000   Number         0  uidiv.o ABSOLUTE
    ../clib/microlib/division.c              0x00000000   Number         0  uldiv.o ABSOLUTE
    ../clib/microlib/init/entry.s            0x00000000   Number         0  entry8b.o ABSOLUTE
    ../clib/microlib/init/entry.s            0x00000000   Number         0  entry11a.o ABSOLUTE
    ../clib/microlib/init/entry.s            0x00000000   Number         0  entry7a.o ABSOLUTE
    ../clib/microlib/init/entry.s            0x00000000   Number         0  entry11b.o ABSOLUTE
    ../clib/microlib/init/entry.s            0x00000000   Number         0  entry9a.o ABSOLUTE
    ../clib/microlib/init/entry.s            0x00000000   Number         0  entry5.o ABSOLUTE
    ../clib/microlib/init/entry.s            0x00000000   Number         0  entry7b.o ABSOLUTE
    ../clib/microlib/init/entry.s            0x00000000   Number         0  entry.o ABSOLUTE
    ../clib/microlib/init/entry.s            0x00000000   Number         0  entry2.o ABSOLUTE
    ../clib/microlib/init/entry.s            0x00000000   Number         0  entry9b.o ABSOLUTE
    ../clib/microlib/init/entry.s            0x00000000   Number         0  entry10a.o ABSOLUTE
    ../clib/microlib/init/entry.s            0x00000000   Number         0  entry8a.o ABSOLUTE
    ../clib/microlib/init/entry.s            0x00000000   Number         0  entry10b.o ABSOLUTE
    ../clib/microlib/longlong.c              0x00000000   Number         0  llsshr.o ABSOLUTE
    ../clib/microlib/longlong.c              0x00000000   Number         0  llushr.o ABSOLUTE
    ../clib/microlib/longlong.c              0x00000000   Number         0  llshl.o ABSOLUTE
    ../clib/microlib/printf/printf.c         0x00000000   Number         0  printf1.o ABSOLUTE
    ../clib/microlib/printf/printf.c         0x00000000   Number         0  printf0.o ABSOLUTE
    ../clib/microlib/printf/printf.c         0x00000000   Number         0  printfb.o ABSOLUTE
    ../clib/microlib/printf/printf.c         0x00000000   Number         0  printf4.o ABSOLUTE
    ../clib/microlib/printf/printf.c         0x00000000   Number         0  printfa.o ABSOLUTE
    ../clib/microlib/printf/printf.c         0x00000000   Number         0  printf8.o ABSOLUTE
    ../clib/microlib/printf/printf.c         0x00000000   Number         0  printf7.o ABSOLUTE
    ../clib/microlib/printf/printf.c         0x00000000   Number         0  printf6.o ABSOLUTE
    ../clib/microlib/printf/printf.c         0x00000000   Number         0  printf5.o ABSOLUTE
    ../clib/microlib/printf/printf.c         0x00000000   Number         0  printf3.o ABSOLUTE
    ../clib/microlib/printf/printf.c         0x00000000   Number         0  printf2.o ABSOLUTE
    ../clib/microlib/printf/stubs.s          0x00000000   Number         0  stubs.o ABSOLUTE
    ../clib/microlib/stdio/streams.c         0x00000000   Number         0  stdout.o ABSOLUTE
    ../clib/microlib/string/memcpy.c         0x00000000   Number         0  memcpyb.o ABSOLUTE
    ../clib/microlib/string/memcpy.c         0x00000000   Number         0  memcpya.o ABSOLUTE
    ../clib/microlib/string/memset.c         0x00000000   Number         0  memseta.o ABSOLUTE
    ../clib/microlib/stubs.s                 0x00000000   Number         0  iusefp.o ABSOLUTE
    ../fplib/microlib/fpadd.c                0x00000000   Number         0  dadd.o ABSOLUTE
    ../fplib/microlib/fpdiv.c                0x00000000   Number         0  ddiv.o ABSOLUTE
    ../fplib/microlib/fpepilogue.c           0x00000000   Number         0  depilogue.o ABSOLUTE
    ../fplib/microlib/fpfix.c                0x00000000   Number         0  dfixul.o ABSOLUTE
    ../fplib/microlib/fpmul.c                0x00000000   Number         0  dmul.o ABSOLUTE
    ..\..\FreeRTOS\croutine.c                0x00000000   Number         0  croutine.o ABSOLUTE
    ..\..\FreeRTOS\event_groups.c            0x00000000   Number         0  event_groups.o ABSOLUTE
    ..\..\FreeRTOS\list.c                    0x00000000   Number         0  list.o ABSOLUTE
    ..\..\FreeRTOS\portable\MemMang\heap_1.c 0x00000000   Number         0  heap_1.o ABSOLUTE
    ..\..\FreeRTOS\portable\RVDS\ARM_CM3\port.c 0x00000000   Number         0  port.o ABSOLUTE
    ..\..\FreeRTOS\queue.c                   0x00000000   Number         0  queue.o ABSOLUTE
    ..\..\FreeRTOS\tasks.c                   0x00000000   Number         0  tasks.o ABSOLUTE
    ..\..\FreeRTOS\timers.c                  0x00000000   Number         0  timers.o ABSOLUTE
    ..\\..\\FreeRTOS\\portable\\RVDS\\ARM_CM3\\port.c 0x00000000   Number         0  port.o ABSOLUTE
    ..\common\basic_io.c                     0x00000000   Number         0  basic_io.o ABSOLUTE
    cdrcmple.s                               0x00000000   Number         0  cdrcmple.o ABSOLUTE
    dc.s                                     0x00000000   Number         0  dc.o ABSOLUTE
    handlers.s                               0x00000000   Number         0  handlers.o ABSOLUTE
    init.s                                   0x00000000   Number         0  init.o ABSOLUTE
    main.c                                   0x00000000   Number         0  main.o ABSOLUTE
    startup_MPS_CM3.s                        0x00000000   Number         0  startup_mps_cm3.o ABSOLUTE
    .ARM.Collect$$$$00000000                 0x000000c0   Section        0  entry.o(.ARM.Collect$$$$00000000)
    .ARM.Collect$$$$00000001                 0x000000c0   Section        4  entry2.o(.ARM.Collect$$$$00000001)
    .ARM.Collect$$$$00000004                 0x000000c4   Section        4  entry5.o(.ARM.Collect$$$$00000004)
    .ARM.Collect$$$$00000008                 0x000000c8   Section        0  entry7b.o(.ARM.Collect$$$$00000008)
    .ARM.Collect$$$$0000000A                 0x000000c8   Section        0  entry8b.o(.ARM.Collect$$$$0000000A)
    .ARM.Collect$$$$0000000B                 0x000000c8   Section        8  entry9a.o(.ARM.Collect$$$$0000000B)
    .ARM.Collect$$$$0000000D                 0x000000d0   Section        0  entry10a.o(.ARM.Collect$$$$0000000D)
    .ARM.Collect$$$$0000000F                 0x000000d0   Section        0  entry11a.o(.ARM.Collect$$$$0000000F)
    .ARM.Collect$$$$00002712                 0x000000d0   Section        4  entry2.o(.ARM.Collect$$$$00002712)
    __lit__00000000                          0x000000d0   Data           4  entry2.o(.ARM.Collect$$$$00002712)
    .emb_text                                0x000000d4   Section      150  port.o(.emb_text)
    .text                                    0x0000016a   Section        0  list.o(.text)
    .text                                    0x00000200   Section        0  queue.o(.text)
    prvInitialiseNewQueue                    0x0000027b   Thumb Code    42  queue.o(.text)
    prvUnlockQueue                           0x000002dd   Thumb Code   126  queue.o(.text)
    prvIsQueueFull                           0x0000035b   Thumb Code    30  queue.o(.text)
    prvCopyDataToQueue                       0x00000379   Thumb Code   124  queue.o(.text)
    prvInitialiseMutex                       0x00000509   Thumb Code    28  queue.o(.text)
    prvIsQueueEmpty                          0x00000649   Thumb Code    26  queue.o(.text)
    prvCopyDataFromQueue                     0x00000663   Thumb Code    42  queue.o(.text)
    .text                                    0x0000096c   Section        0  tasks.o(.text)
    prvInitialiseTaskLists                   0x0000096d   Thumb Code    64  tasks.o(.text)
    prvAddNewTaskToReadyList                 0x000009ad   Thumb Code   156  tasks.o(.text)
    prvInitialiseNewTask                     0x00000a49   Thumb Code   144  tasks.o(.text)
    prvResetNextTaskUnblockTime              0x00000b39   Thumb Code    42  tasks.o(.text)
    prvAddCurrentTaskToDelayedList           0x00000d15   Thumb Code   202  tasks.o(.text)
    prvTaskIsTaskSuspended                   0x00000fd3   Thumb Code    56  tasks.o(.text)
    prvCheckTasksWaitingTermination          0x000010f5   Thumb Code     2  tasks.o(.text)
    prvIdleTask                              0x000010f7   Thumb Code     8  tasks.o(.text)
    prvTaskCheckFreeStackSpace               0x000011e5   Thumb Code    22  tasks.o(.text)
    prvListTasksWithinSingleList             0x0000126d   Thumb Code   106  tasks.o(.text)
    .text                                    0x00001a30   Section        0  timers.o(.text)
    prvInsertTimerInActiveList               0x00001a31   Thumb Code    80  timers.o(.text)
    prvSwitchTimerLists                      0x00001ae7   Thumb Code   122  timers.o(.text)
    prvSampleTimeNow                         0x00001b61   Thumb Code    40  timers.o(.text)
    prvProcessReceivedCommands               0x00001b89   Thumb Code   184  timers.o(.text)
    prvProcessExpiredTimer                   0x00001c41   Thumb Code    70  timers.o(.text)
    prvProcessTimerOrBlockTask               0x00001c87   Thumb Code   102  timers.o(.text)
    prvGetNextExpireTime                     0x00001ced   Thumb Code    36  timers.o(.text)
    prvTimerTask                             0x00001d11   Thumb Code    26  timers.o(.text)
    prvCheckForValidListAndQueue             0x00001d2b   Thumb Code    56  timers.o(.text)
    prvInitialiseNewTimer                    0x00001d8b   Thumb Code    46  timers.o(.text)
    .text                                    0x00001e7c   Section        0  heap_1.o(.text)
    .text                                    0x00001f00   Section        0  port.o(.text)
    prvTaskExitError                         0x00001f01   Thumb Code    22  port.o(.text)
    .text                                    0x00001fe8   Section        0  main.o(.text)
    .text                                    0x000020d8   Section        0  basic_io.o(.text)
    .text                                    0x00002130   Section       28  startup_mps_cm3.o(.text)
    .text                                    0x0000214c   Section        0  memcpya.o(.text)
    .text                                    0x00002170   Section        0  memseta.o(.text)
    .text                                    0x00002194   Section        0  uidiv.o(.text)
    .text                                    0x000021c0   Section       36  init.o(.text)
    i.__0printf$3                            0x000021e4   Section        0  printf3.o(i.__0printf$3)
    i.__scatterload_copy                     0x00002204   Section       14  handlers.o(i.__scatterload_copy)
    i.__scatterload_null                     0x00002212   Section        2  handlers.o(i.__scatterload_null)
    i.__scatterload_zeroinit                 0x00002214   Section       14  handlers.o(i.__scatterload_zeroinit)
    i._printf_core                           0x00002224   Section        0  printf3.o(i._printf_core)
    _printf_core                             0x00002225   Thumb Code   436  printf3.o(i._printf_core)
    .bss                                     0x10000000   Section     4096  heap_1.o(.bss)
    ucHeap                                   0x10000000   Data        4096  heap_1.o(.bss)
    .data                                    0x2007c000   Section       56  tasks.o(.data)
    pxDelayedTaskList                        0x2007c004   Data           4  tasks.o(.data)
    pxOverflowDelayedTaskList                0x2007c008   Data           4  tasks.o(.data)
    uxCurrentNumberOfTasks                   0x2007c00c   Data           4  tasks.o(.data)
    xTickCount                               0x2007c010   Data           4  tasks.o(.data)
    uxTopReadyPriority                       0x2007c014   Data           4  tasks.o(.data)
    xSchedulerRunning                        0x2007c018   Data           4  tasks.o(.data)
    uxPendedTicks                            0x2007c01c   Data           4  tasks.o(.data)
    xYieldPending                            0x2007c020   Data           4  tasks.o(.data)
    xNumOfOverflows                          0x2007c024   Data           4  tasks.o(.data)
    uxTaskNumber                             0x2007c028   Data           4  tasks.o(.data)
    xNextTaskUnblockTime                     0x2007c02c   Data           4  tasks.o(.data)
    xIdleTaskHandle                          0x2007c030   Data           4  tasks.o(.data)
    uxSchedulerSuspended                     0x2007c034   Data           4  tasks.o(.data)
    .data                                    0x2007c038   Section       20  timers.o(.data)
    pxCurrentTimerList                       0x2007c038   Data           4  timers.o(.data)
    pxOverflowTimerList                      0x2007c03c   Data           4  timers.o(.data)
    xTimerQueue                              0x2007c040   Data           4  timers.o(.data)
    xTimerTaskHandle                         0x2007c044   Data           4  timers.o(.data)
    xLastTime                                0x2007c048   Data           4  timers.o(.data)
    .data                                    0x2007c04c   Section        8  heap_1.o(.data)
    xNextFreeByte                            0x2007c04c   Data           4  heap_1.o(.data)
    pucAlignedHeap                           0x2007c050   Data           4  heap_1.o(.data)
    .data                                    0x2007c054   Section        4  port.o(.data)
    uxCriticalNesting                        0x2007c054   Data           4  port.o(.data)
    .data                                    0x2007c058   Section       16  main.o(.data)
    .data                                    0x2007c068   Section        4  stdout.o(.data)
    .bss                                     0x2007c06c   Section      180  tasks.o(.bss)
    pxReadyTasksLists                        0x2007c06c   Data         100  tasks.o(.bss)
    xDelayedTaskList1                        0x2007c0d0   Data          20  tasks.o(.bss)
    xDelayedTaskList2                        0x2007c0e4   Data          20  tasks.o(.bss)
    xPendingReadyList                        0x2007c0f8   Data          20  tasks.o(.bss)
    xSuspendedTaskList                       0x2007c10c   Data          20  tasks.o(.bss)
    .bss                                     0x2007c120   Section       40  timers.o(.bss)
    xActiveTimerList1                        0x2007c120   Data          20  timers.o(.bss)
    xActiveTimerList2                        0x2007c134   Data          20  timers.o(.bss)
    .bss                                     0x2007c148   Section       12  main.o(.bss)
    STACK                                    0x2007c158   Section      512  startup_mps_cm3.o(STACK)

    Global Symbols

    Symbol Name                              Value     Ov Type        Size  Object(Section)

    BuildAttributes$$THM_ISAv4$P$D$K$B$S$PE$A:L22UL41UL21$X:L11$S22US41US21$IEEE1$IW$USESV6$~STKCKD$USESV7$~SHL$OSPACE$ROPI$EBA8$MICROLIB$REQ8$PRES8$EABIv2 0x00000000   Number         0  anon$$obj.o ABSOLUTE
    __ARM_use_no_argv                        0x00000000   Number         0  main.o ABSOLUTE
    __Vectors                                0x00000000   Data           4  startup_mps_cm3.o(RESET)
    _printf_a                                0x00000000   Number         0  stubs.o ABSOLUTE
    _printf_c                                0x00000000   Number         0  stubs.o ABSOLUTE
    _printf_charcount                        0x00000000   Number         0  stubs.o ABSOLUTE
    _printf_d                                0x00000000   Number         0  stubs.o ABSOLUTE
    _printf_e                                0x00000000   Number         0  stubs.o ABSOLUTE
    _printf_f                                0x00000000   Number         0  stubs.o ABSOLUTE
    _printf_flags                            0x00000000   Number         0  stubs.o ABSOLUTE
    _printf_fp_dec                           0x00000000   Number         0  stubs.o ABSOLUTE
    _printf_fp_hex                           0x00000000   Number         0  stubs.o ABSOLUTE
    _printf_g                                0x00000000   Number         0  stubs.o ABSOLUTE
    _printf_i                                0x00000000   Number         0  stubs.o ABSOLUTE
    _printf_int_dec                          0x00000000   Number         0  stubs.o ABSOLUTE
    _printf_l                                0x00000000   Number         0  stubs.o ABSOLUTE
    _printf_lc                               0x00000000   Number         0  stubs.o ABSOLUTE
    _printf_ll                               0x00000000   Number         0  stubs.o ABSOLUTE
    _printf_lld                              0x00000000   Number         0  stubs.o ABSOLUTE
    _printf_lli                              0x00000000   Number         0  stubs.o ABSOLUTE
    _printf_llo                              0x00000000   Number         0  stubs.o ABSOLUTE
    _printf_llu                              0x00000000   Number         0  stubs.o ABSOLUTE
    _printf_llx                              0x00000000   Number         0  stubs.o ABSOLUTE
    _printf_longlong_dec                     0x00000000   Number         0  stubs.o ABSOLUTE
    _printf_longlong_hex                     0x00000000   Number         0  stubs.o ABSOLUTE
    _printf_longlong_oct                     0x00000000   Number         0  stubs.o ABSOLUTE
    _printf_ls                               0x00000000   Number         0  stubs.o ABSOLUTE
    _printf_mbtowc                           0x00000000   Number         0  stubs.o ABSOLUTE
    _printf_n                                0x00000000   Number         0  stubs.o ABSOLUTE
    _printf_o                                0x00000000   Number         0  stubs.o ABSOLUTE
    _printf_p                                0x00000000   Number         0  stubs.o ABSOLUTE
    _printf_percent                          0x00000000   Number         0  stubs.o ABSOLUTE
    _printf_pre_padding                      0x00000000   Number         0  stubs.o ABSOLUTE
    _printf_return_value                     0x00000000   Number         0  stubs.o ABSOLUTE
    _printf_s                                0x00000000   Number         0  stubs.o ABSOLUTE
    _printf_sizespec                         0x00000000   Number         0  stubs.o ABSOLUTE
    _printf_str                              0x00000000   Number         0  stubs.o ABSOLUTE
    _printf_truncate_signed                  0x00000000   Number         0  stubs.o ABSOLUTE
    _printf_truncate_unsigned                0x00000000   Number         0  stubs.o ABSOLUTE
    _printf_u                                0x00000000   Number         0  stubs.o ABSOLUTE
    _printf_wc                               0x00000000   Number         0  stubs.o ABSOLUTE
    _printf_wctomb                           0x00000000   Number         0  stubs.o ABSOLUTE
    _printf_widthprec                        0x00000000   Number         0  stubs.o ABSOLUTE
    _printf_x                                0x00000000   Number         0  stubs.o ABSOLUTE
    __cpp_initialize__aeabi_                  - Undefined Weak Reference
    __cxa_finalize                            - Undefined Weak Reference
    __decompress                              - Undefined Weak Reference
    _clock_init                               - Undefined Weak Reference
    _microlib_exit                            - Undefined Weak Reference
    __main                                   0x000000c1   Thumb Code     0  entry.o(.ARM.Collect$$$$00000000)
    _main_stk                                0x000000c1   Thumb Code     0  entry2.o(.ARM.Collect$$$$00000001)
    _main_scatterload                        0x000000c5   Thumb Code     0  entry5.o(.ARM.Collect$$$$00000004)
    __main_after_scatterload                 0x000000c9   Thumb Code     0  entry5.o(.ARM.Collect$$$$00000004)
    _main_clock                              0x000000c9   Thumb Code     0  entry7b.o(.ARM.Collect$$$$00000008)
    _main_cpp_init                           0x000000c9   Thumb Code     0  entry8b.o(.ARM.Collect$$$$0000000A)
    _main_init                               0x000000c9   Thumb Code     0  entry9a.o(.ARM.Collect$$$$0000000B)
    __rt_final_cpp                           0x000000d1   Thumb Code     0  entry10a.o(.ARM.Collect$$$$0000000D)
    __rt_final_exit                          0x000000d1   Thumb Code     0  entry11a.o(.ARM.Collect$$$$0000000F)
    vPortSVCHandler                          0x000000d5   Thumb Code    32  port.o(.emb_text)
    __asm___6_port_c_39a90d8d__prvStartFirstTask 0x000000f9   Thumb Code    28  port.o(.emb_text)
    xPortPendSVHandler                       0x00000119   Thumb Code    72  port.o(.emb_text)
    vPortGetIPSR                             0x00000165   Thumb Code     6  port.o(.emb_text)
    vListInitialise                          0x0000016b   Thumb Code    26  list.o(.text)
    vListInitialiseItem                      0x00000185   Thumb Code     6  list.o(.text)
    vListInsertEnd                           0x0000018b   Thumb Code    24  list.o(.text)
    vListInsert                              0x000001a3   Thumb Code    52  list.o(.text)
    uxListRemove                             0x000001d7   Thumb Code    40  list.o(.text)
    xQueueGenericReset                       0x00000201   Thumb Code   122  queue.o(.text)
    xQueueGenericCreate                      0x000002a5   Thumb Code    56  queue.o(.text)
    xQueueGenericSend                        0x000003f5   Thumb Code   276  queue.o(.text)
    xQueueCreateMutex                        0x00000525   Thumb Code    34  queue.o(.text)
    xQueueGenericSendFromISR                 0x00000547   Thumb Code   134  queue.o(.text)
    xQueueGiveFromISR                        0x000005cd   Thumb Code   124  queue.o(.text)
    xQueueGenericReceive                     0x0000068d   Thumb Code   342  queue.o(.text)
    xQueueReceiveFromISR                     0x000007e3   Thumb Code   130  queue.o(.text)
    xQueuePeekFromISR                        0x00000865   Thumb Code    74  queue.o(.text)
    uxQueueMessagesWaiting                   0x000008af   Thumb Code    18  queue.o(.text)
    uxQueueSpacesAvailable                   0x000008c1   Thumb Code    24  queue.o(.text)
    uxQueueMessagesWaitingFromISR            0x000008d9   Thumb Code     6  queue.o(.text)
    vQueueDelete                             0x000008df   Thumb Code    14  queue.o(.text)
    uxQueueGetQueueNumber                    0x000008ed   Thumb Code     6  queue.o(.text)
    vQueueSetQueueNumber                     0x000008f3   Thumb Code     4  queue.o(.text)
    ucQueueGetQueueType                      0x000008f7   Thumb Code     8  queue.o(.text)
    xQueueIsQueueEmptyFromISR                0x000008ff   Thumb Code    14  queue.o(.text)
    xQueueIsQueueFullFromISR                 0x0000090d   Thumb Code    18  queue.o(.text)
    vQueueWaitForMessageRestricted           0x0000091f   Thumb Code    74  queue.o(.text)
    xTaskCreate                              0x00000ad9   Thumb Code    96  tasks.o(.text)
    xTaskIncrementTick                       0x00000b63   Thumb Code   238  tasks.o(.text)
    xTaskResumeAll                           0x00000c51   Thumb Code   196  tasks.o(.text)
    vTaskSuspendAll                          0x00000ddf   Thumb Code    12  tasks.o(.text)
    vTaskDelayUntil                          0x00000deb   Thumb Code   106  tasks.o(.text)
    vTaskDelay                               0x00000e55   Thumb Code    46  tasks.o(.text)
    eTaskGetState                            0x00000e83   Thumb Code    76  tasks.o(.text)
    vTaskSwitchContext                       0x00000ecf   Thumb Code   100  tasks.o(.text)
    vTaskSuspend                             0x00000f33   Thumb Code   160  tasks.o(.text)
    vTaskResume                              0x0000100b   Thumb Code   104  tasks.o(.text)
    xTaskResumeFromISR                       0x00001073   Thumb Code   130  tasks.o(.text)
    vTaskStartScheduler                      0x000010ff   Thumb Code    82  tasks.o(.text)
    vTaskEndScheduler                        0x00001151   Thumb Code    32  tasks.o(.text)
    xTaskGetTickCount                        0x00001171   Thumb Code     6  tasks.o(.text)
    xTaskGetTickCountFromISR                 0x00001177   Thumb Code     8  tasks.o(.text)
    uxTaskGetNumberOfTasks                   0x0000117f   Thumb Code    82  tasks.o(.text)
    pcTaskGetName                            0x000011d1   Thumb Code    20  tasks.o(.text)
    vTaskGetInfo                             0x000011fb   Thumb Code   114  tasks.o(.text)
    uxTaskGetSystemState                     0x000012d7   Thumb Code   134  tasks.o(.text)
    vTaskPlaceOnEventList                    0x0000135d   Thumb Code    28  tasks.o(.text)
    vTaskPlaceOnUnorderedEventList           0x00001379   Thumb Code    40  tasks.o(.text)
    vTaskPlaceOnEventListRestricted          0x000013a1   Thumb Code    36  tasks.o(.text)
    xTaskRemoveFromEventList                 0x000013c5   Thumb Code   104  tasks.o(.text)
    xTaskRemoveFromUnorderedEventList        0x0000142d   Thumb Code    94  tasks.o(.text)
    vTaskSetTimeOutState                     0x0000148b   Thumb Code    14  tasks.o(.text)
    xTaskCheckForTimeOut                     0x00001499   Thumb Code    84  tasks.o(.text)
    vTaskMissedYield                         0x000014ed   Thumb Code     8  tasks.o(.text)
    uxTaskGetTaskNumber                      0x000014f5   Thumb Code    14  tasks.o(.text)
    vTaskSetTaskNumber                       0x00001503   Thumb Code     8  tasks.o(.text)
    xTaskGetCurrentTaskHandle                0x0000150b   Thumb Code     6  tasks.o(.text)
    xTaskGetSchedulerState                   0x00001511   Thumb Code    24  tasks.o(.text)
    vTaskPriorityInherit                     0x00001529   Thumb Code   218  tasks.o(.text)
    xTaskPriorityDisinherit                  0x00001603   Thumb Code   122  tasks.o(.text)
    uxTaskResetEventItemValue                0x0000167d   Thumb Code    24  tasks.o(.text)
    pvTaskIncrementMutexHeldCount            0x00001695   Thumb Code    26  tasks.o(.text)
    ulTaskNotifyTake                         0x000016af   Thumb Code   108  tasks.o(.text)
    xTaskNotifyWait                          0x0000171b   Thumb Code   150  tasks.o(.text)
    xTaskGenericNotify                       0x000017b1   Thumb Code   178  tasks.o(.text)
    xTaskGenericNotifyFromISR                0x00001863   Thumb Code   228  tasks.o(.text)
    vTaskNotifyGiveFromISR                   0x00001947   Thumb Code   182  tasks.o(.text)
    xTaskNotifyStateClear                    0x000019fd   Thumb Code    48  tasks.o(.text)
    xTimerGenericCommand                     0x00001a81   Thumb Code   102  timers.o(.text)
    xTimerCreateTimerTask                    0x00001d63   Thumb Code    40  timers.o(.text)
    xTimerCreate                             0x00001db9   Thumb Code    48  timers.o(.text)
    xTimerGetTimerDaemonTaskHandle           0x00001de9   Thumb Code     6  timers.o(.text)
    xTimerGetPeriod                          0x00001def   Thumb Code     8  timers.o(.text)
    xTimerGetExpiryTime                      0x00001df7   Thumb Code     8  timers.o(.text)
    pcTimerGetName                           0x00001dff   Thumb Code     8  timers.o(.text)
    xTimerIsTimerActive                      0x00001e07   Thumb Code    32  timers.o(.text)
    pvTimerGetTimerID                        0x00001e27   Thumb Code    66  timers.o(.text)
    vTimerSetTimerID                         0x00001e69   Thumb Code    20  timers.o(.text)
    pvPortMalloc                             0x00001e7d   Thumb Code    98  heap_1.o(.text)
    vPortFree                                0x00001edf   Thumb Code     2  heap_1.o(.text)
    vPortInitialiseBlocks                    0x00001ee1   Thumb Code     8  heap_1.o(.text)
    xPortGetFreeHeapSize                     0x00001ee9   Thumb Code    12  heap_1.o(.text)
    pxPortInitialiseStack                    0x00001f17   Thumb Code    30  port.o(.text)
    vPortSetupTimerInterrupt                 0x00001f35   Thumb Code    16  port.o(.text)
    xPortStartScheduler                      0x00001f45   Thumb Code    42  port.o(.text)
    vPortEndScheduler                        0x00001f6f   Thumb Code     2  port.o(.text)
    vPortEnterCritical                       0x00001f71   Thumb Code    30  port.o(.text)
    vPortExitCritical                        0x00001f8f   Thumb Code    28  port.o(.text)
    xPortSysTickHandler                      0x00001fab   Thumb Code    48  port.o(.text)
    vTimerCallback                           0x00001fe9   Thumb Code    40  main.o(.text)
    main                                     0x00002011   Thumb Code   104  main.o(.text)
    vPrintString                             0x000020d9   Thumb Code    20  basic_io.o(.text)
    vPrintStringAndNumber                    0x000020ed   Thumb Code    26  basic_io.o(.text)
    fputc                                    0x00002107   Thumb Code    30  basic_io.o(.text)
    Reset_Handler                            0x00002131   Thumb Code     4  startup_mps_cm3.o(.text)
    NMI_Handler                              0x00002135   Thumb Code     2  startup_mps_cm3.o(.text)
    HardFault_Handler                        0x00002137   Thumb Code     2  startup_mps_cm3.o(.text)
    MemManage_Handler                        0x00002139   Thumb Code     2  startup_mps_cm3.o(.text)
    BusFault_Handler                         0x0000213b   Thumb Code     2  startup_mps_cm3.o(.text)
    UsageFault_Handler                       0x0000213d   Thumb Code     2  startup_mps_cm3.o(.text)
    SVC_Handler                              0x0000213f   Thumb Code     2  startup_mps_cm3.o(.text)
    DebugMon_Handler                         0x00002141   Thumb Code     2  startup_mps_cm3.o(.text)
    PendSV_Handler                           0x00002143   Thumb Code     2  startup_mps_cm3.o(.text)
    SysTick_Handler                          0x00002145   Thumb Code     2  startup_mps_cm3.o(.text)
    AACI_IRQHandler                          0x00002147   Thumb Code     0  startup_mps_cm3.o(.text)
    CAN_IRQHandler                           0x00002147   Thumb Code     0  startup_mps_cm3.o(.text)
    CHLCD_IRQHandler                         0x00002147   Thumb Code     0  startup_mps_cm3.o(.text)
    CLCD_IRQHandler                          0x00002147   Thumb Code     0  startup_mps_cm3.o(.text)
    CPU_CLCD_IRQHandler                      0x00002147   Thumb Code     0  startup_mps_cm3.o(.text)
    ENET_IRQHandler                          0x00002147   Thumb Code     0  startup_mps_cm3.o(.text)
    FLEXRAY_IRQHandler                       0x00002147   Thumb Code     0  startup_mps_cm3.o(.text)
    I2C_IRQHandler                           0x00002147   Thumb Code     0  startup_mps_cm3.o(.text)
    LIN_IRQHandler                           0x00002147   Thumb Code     0  startup_mps_cm3.o(.text)
    MCIA_IRQHandler                          0x00002147   Thumb Code     0  startup_mps_cm3.o(.text)
    MCIB_IRQHandler                          0x00002147   Thumb Code     0  startup_mps_cm3.o(.text)
    RTC_IRQHandler                           0x00002147   Thumb Code     0  startup_mps_cm3.o(.text)
    SPI_IRQHandler                           0x00002147   Thumb Code     0  startup_mps_cm3.o(.text)
    TIM0_IRQHandler                          0x00002147   Thumb Code     0  startup_mps_cm3.o(.text)
    TIM2_IRQHandler                          0x00002147   Thumb Code     0  startup_mps_cm3.o(.text)
    UART0_IRQHandler                         0x00002147   Thumb Code     0  startup_mps_cm3.o(.text)
    UART1_IRQHandler                         0x00002147   Thumb Code     0  startup_mps_cm3.o(.text)
    UART2_IRQHandler                         0x00002147   Thumb Code     0  startup_mps_cm3.o(.text)
    UART3_IRQHandler                         0x00002147   Thumb Code     0  startup_mps_cm3.o(.text)
    UART4_IRQHandler                         0x00002147   Thumb Code     0  startup_mps_cm3.o(.text)
    USBDC_IRQHandler                         0x00002147   Thumb Code     0  startup_mps_cm3.o(.text)
    USBHC_IRQHandler                         0x00002147   Thumb Code     0  startup_mps_cm3.o(.text)
    WDT_IRQHandler                           0x00002147   Thumb Code     0  startup_mps_cm3.o(.text)
    __aeabi_memcpy                           0x0000214d   Thumb Code    36  memcpya.o(.text)
    __aeabi_memcpy4                          0x0000214d   Thumb Code     0  memcpya.o(.text)
    __aeabi_memcpy8                          0x0000214d   Thumb Code     0  memcpya.o(.text)
    __aeabi_memset                           0x00002171   Thumb Code    14  memseta.o(.text)
    __aeabi_memset4                          0x00002171   Thumb Code     0  memseta.o(.text)
    __aeabi_memset8                          0x00002171   Thumb Code     0  memseta.o(.text)
    __aeabi_memclr                           0x0000217f   Thumb Code     4  memseta.o(.text)
    __aeabi_memclr4                          0x0000217f   Thumb Code     0  memseta.o(.text)
    __aeabi_memclr8                          0x0000217f   Thumb Code     0  memseta.o(.text)
    _memset$wrapper                          0x00002183   Thumb Code    18  memseta.o(.text)
    __aeabi_uidiv                            0x00002195   Thumb Code     0  uidiv.o(.text)
    __aeabi_uidivmod                         0x00002195   Thumb Code    44  uidiv.o(.text)
    __scatterload                            0x000021c1   Thumb Code    28  init.o(.text)
    __scatterload_rt2                        0x000021c1   Thumb Code     0  init.o(.text)
    __0printf$3                              0x000021e5   Thumb Code    22  printf3.o(i.__0printf$3)
    __1printf$3                              0x000021e5   Thumb Code     0  printf3.o(i.__0printf$3)
    __2printf                                0x000021e5   Thumb Code     0  printf3.o(i.__0printf$3)
    __scatterload_copy                       0x00002205   Thumb Code    14  handlers.o(i.__scatterload_copy)
    __scatterload_null                       0x00002213   Thumb Code     2  handlers.o(i.__scatterload_null)
    __scatterload_zeroinit                   0x00002215   Thumb Code    14  handlers.o(i.__scatterload_zeroinit)
    Region$$Table$$Base                      0x000023dc   Number         0  anon$$obj.o(Region$$Table)
    Region$$Table$$Limit                     0x0000240c   Number         0  anon$$obj.o(Region$$Table)
    pxCurrentTCB                             0x2007c000   Data           4  tasks.o(.data)
    xTimers                                  0x2007c058   Data           8  main.o(.data)
    ulLed                                    0x2007c060   Data           8  main.o(.data)
    __stdout                                 0x2007c068   Data           4  stdout.o(.data)
    ulTaskNumber                             0x2007c148   Data          12  main.o(.bss)
    __initial_sp                             0x2007c358   Data           0  startup_mps_cm3.o(STACK)



==============================================================================

Memory Map of the image

  Image Entry point : 0x000000c1

  Load Region LR_IROM1 (Base: 0x00000000, Size: 0x00002478, Max: 0x00080000, ABSOLUTE)

    Execution Region ER_IROM1 (Exec base: 0x00000000, Load base: 0x00000000, Size: 0x0000240c, Max: 0x00080000, ABSOLUTE)

    Exec Addr    Load Addr    Size         Type   Attr      Idx    E Section Name        Object

    0x00000000   0x00000000   0x000000c0   Data   RO          253    RESET               startup_mps_cm3.o
    0x000000c0   0x000000c0   0x00000000   Code   RO          258  * .ARM.Collect$$$$00000000  mc_w.l(entry.o)
    0x000000c0   0x000000c0   0x00000004   Code   RO          528    .ARM.Collect$$$$00000001  mc_w.l(entry2.o)
    0x000000c4   0x000000c4   0x00000004   Code   RO          531    .ARM.Collect$$$$00000004  mc_w.l(entry5.o)
    0x000000c8   0x000000c8   0x00000000   Code   RO          533    .ARM.Collect$$$$00000008  mc_w.l(entry7b.o)
    0x000000c8   0x000000c8   0x00000000   Code   RO          535    .ARM.Collect$$$$0000000A  mc_w.l(entry8b.o)
    0x000000c8   0x000000c8   0x00000008   Code   RO          536    .ARM.Collect$$$$0000000B  mc_w.l(entry9a.o)
    0x000000d0   0x000000d0   0x00000000   Code   RO          538    .ARM.Collect$$$$0000000D  mc_w.l(entry10a.o)
    0x000000d0   0x000000d0   0x00000000   Code   RO          540    .ARM.Collect$$$$0000000F  mc_w.l(entry11a.o)
    0x000000d0   0x000000d0   0x00000004   Code   RO          529    .ARM.Collect$$$$00002712  mc_w.l(entry2.o)
    0x000000d4   0x000000d4   0x00000096   Code   RO          176    .emb_text           port.o
    0x0000016a   0x0000016a   0x00000094   Code   RO           85    .text               list.o
    0x000001fe   0x000001fe   0x00000002   PAD
    0x00000200   0x00000200   0x0000076c   Code   RO           97    .text               queue.o
    0x0000096c   0x0000096c   0x000010c4   Code   RO          115    .text               tasks.o
    0x00001a30   0x00001a30   0x0000044c   Code   RO          146    .text               timers.o
    0x00001e7c   0x00001e7c   0x00000084   Code   RO          161    .text               heap_1.o
    0x00001f00   0x00001f00   0x000000e8   Code   RO          177    .text               port.o
    0x00001fe8   0x00001fe8   0x000000f0   Code   RO          207    .text               main.o
    0x000020d8   0x000020d8   0x00000058   Code   RO          229    .text               basic_io.o
    0x00002130   0x00002130   0x0000001c   Code   RO          254    .text               startup_mps_cm3.o
    0x0000214c   0x0000214c   0x00000024   Code   RO          261    .text               mc_w.l(memcpya.o)
    0x00002170   0x00002170   0x00000024   Code   RO          263    .text               mc_w.l(memseta.o)
    0x00002194   0x00002194   0x0000002c   Code   RO          543    .text               mc_w.l(uidiv.o)
    0x000021c0   0x000021c0   0x00000024   Code   RO          558    .text               mc_w.l(init.o)
    0x000021e4   0x000021e4   0x00000020   Code   RO          356    i.__0printf$3       mc_w.l(printf3.o)
    0x00002204   0x00002204   0x0000000e   Code   RO          570    i.__scatterload_copy  mc_w.l(handlers.o)
    0x00002212   0x00002212   0x00000002   Code   RO          571    i.__scatterload_null  mc_w.l(handlers.o)
    0x00002214   0x00002214   0x0000000e   Code   RO          572    i.__scatterload_zeroinit  mc_w.l(handlers.o)
    0x00002222   0x00002222   0x00000002   PAD
    0x00002224   0x00002224   0x000001b8   Code   RO          363    i._printf_core      mc_w.l(printf3.o)
    0x000023dc   0x000023dc   0x00000030   Data   RO          568    Region$$Table       anon$$obj.o


    Execution Region RW_IRAM1 (Exec base: 0x10000000, Load base: 0x0000240c, Size: 0x00001000, Max: 0x00008000, ABSOLUTE)

    Exec Addr    Load Addr    Size         Type   Attr      Idx    E Section Name        Object

    0x10000000        -       0x00001000   Zero   RW          162    .bss                heap_1.o


    Execution Region RW_IRAM2 (Exec base: 0x2007c000, Load base: 0x0000240c, Size: 0x00000358, Max: 0x00008000, ABSOLUTE)

    Exec Addr    Load Addr    Size         Type   Attr      Idx    E Section Name        Object

    0x2007c000   0x0000240c   0x00000038   Data   RW          117    .data               tasks.o
    0x2007c038   0x00002444   0x00000014   Data   RW          148    .data               timers.o
    0x2007c04c   0x00002458   0x00000008   Data   RW          163    .data               heap_1.o
    0x2007c054   0x00002460   0x00000004   Data   RW          178    .data               port.o
    0x2007c058   0x00002464   0x00000010   Data   RW          209    .data               main.o
    0x2007c068   0x00002474   0x00000004   Data   RW          542    .data               mc_w.l(stdout.o)
    0x2007c06c        -       0x000000b4   Zero   RW          116    .bss                tasks.o
    0x2007c120        -       0x00000028   Zero   RW          147    .bss                timers.o
    0x2007c148        -       0x0000000c   Zero   RW          208    .bss                main.o
    0x2007c154   0x00002478   0x00000004   PAD
    0x2007c158        -       0x00000200   Zero   RW          251    STACK               startup_mps_cm3.o


==============================================================================

Image component sizes


      Code (inc. data)   RO Data    RW Data    ZI Data      Debug   Object Name

        88         12          0          0          0       2211   basic_io.o
         0          0          0          0          0      14532   croutine.o
         0          0          0          0          0      11772   event_groups.o
       132         12          0          8       4096       1960   heap_1.o
       148          0          0          0          0       1854   list.o
       240         96          0         16         12       1423   main.o
       382         26          0          4          0       7076   port.o
      1900          8          0          0          0      14538   queue.o
        28          4        192          0        512        760   startup_mps_cm3.o
      4292        248          0         56        180      28850   tasks.o
      1100         56          0         20         40       7747   timers.o

    ----------------------------------------------------------------------
      8312        462        240        104       4844      92723   Object Totals
         0          0         48          0          0          0   (incl. Generated)
         2          0          0          0          4          0   (incl. Padding)

    ----------------------------------------------------------------------

      Code (inc. data)   RO Data    RW Data    ZI Data      Debug   Library Member Name

         0          0          0          0          0          0   entry.o
         0          0          0          0          0          0   entry10a.o
         0          0          0          0          0          0   entry11a.o
         8          4          0          0          0          0   entry2.o
         4          0          0          0          0          0   entry5.o
         0          0          0          0          0          0   entry7b.o
         0          0          0          0          0          0   entry8b.o
         8          4          0          0          0          0   entry9a.o
        30          0          0          0          0          0   handlers.o
        36          8          0          0          0         68   init.o
        36          0          0          0          0         68   memcpya.o
        36          0          0          0          0        108   memseta.o
       472         14          0          0          0        184   printf3.o
         0          0          0          4          0          0   stdout.o
        44          0          0          0          0         80   uidiv.o

    ----------------------------------------------------------------------
       676         30          0          4          0        508   Library Totals
         2          0          0          0          0          0   (incl. Padding)

    ----------------------------------------------------------------------

      Code (inc. data)   RO Data    RW Data    ZI Data      Debug   Library Name

       674         30          0          4          0        508   mc_w.l

    ----------------------------------------------------------------------
       676         30          0          4          0        508   Library Totals

    ----------------------------------------------------------------------

==============================================================================


      Code (inc. data)   RO Data    RW Data    ZI Data      Debug   

      8988        492        240        108       4844      92291   Grand Totals
      8988        492        240        108       4844      92291   ELF Image Totals
      8988        492        240        108          0          0   ROM Totals

==============================================================================

    Total RO  Size (Code + RO Data)                 9228 (   9.01kB)
    Total RW  Size (RW Data + ZI Data)              4952 (   4.84kB)
    Total ROM Size (Code + RO Data + RW Data)       9336 (   9.12kB)

==============================================================================

